:020000020000FC
:10000000C4CD00000000000020C0AEC18EC00000C2
:10001000000098C000000000000000000203040679
:10002000080C10182030406080000406080C1018DE
:100030002030406080A0C0000003070F1F000D0D9E
:1000400004050D050305030302004FB662FD0CC055
:10005000552041F00994C52DC095089483FDC7959E
:10006000C4BD64604FBE1895C0916400089483FDC0
:10007000C795C4BD6B7FC0916400CF3F09F41EC01B
:1000800070FF1AC082FD05C04FBEAC98929894983C
:10009000189576FD0EC064FD0CC0C091B100C0FD86
:1000A0009598C1FDAD98C2FD9398CAEFC095CA95C9
:1000B000F1F7AC98929894984FBE189524BCCC2731
:1000C000C064C8BF6460F8CFC6CF70FFC4CF64FD02
:1000D000C2CFAC9AC0CF70FFBECF64FDBCCF929AA6
:1000E000BACF70FFB8CF64FDB6CF949AB4CF959ACB
:1000F00070FFB1CF64FDAFCFC7E0CA95F1F7AC9AFE
:10010000AACFAD9A70FFA7CF64FDA5CFC7E0CA956F
:10011000F1F7929AA0CF939A70FF9DCF64FD9BCF89
:10012000C7E0CA95F1F7949A96CF4FB6C9B7CF7E7C
:10013000C9BF6E7FCCB5CE0DDDB5DF1DDBBDCABD41
:100140004FBE18953FB68F7EA9B7A072A2118061ED
:10015000A9B7AF7DA9BFA9B7AE7FA9BF7894A09179
:100160006800AA2341F085FD2FC0A0916800AA95E0
:10017000A093680029C040E050E085FD15C0A6B3FB
:1001800096FDA095A0FD4FEFAEB5A06496FDAF7BA8
:10019000AEBDAA27A062A8BF8D7FA6B396FDA0958D
:1001A000A0FD5FEF451739F7A8E161FDA093680056
:1001B00085FD03C0A8E1A09368004093960081608C
:1001C000442311F02092990085FD0EC0A091690092
:1001D000AA2331F0A0916900AA95A093690004C0F8
:1001E0008061AA27A062A8BF80FF3CC0A0919600B2
:1001F0004A2F61FF8E7F85FD1CC0A091B400A43002
:10020000C1F4403F08F040EFA42FA295AF704A0F11
:100210005091B600533069F0A695A69550FD01C0E7
:10022000A69552FD03C0A41B4A2F03C04A0F08F431
:100230004FEF40936100A72FA670A1F073FD12C08D
:10024000A0917000AA0FAA0F50919E005695569546
:10025000541708F0452F4A0F4093610018F4AFEF90
:10026000A09361004091B400443009F03EC0A091D9
:100270006100A093630040916300A0919B004A1726
:1002800008F04A2FA0919D004A1708F04A2F542EDB
:10029000A091A000AA2309F422C0542F5A1B10F4E5
:1002A000A42F50E0BA2E8894AA1FAA2EA091A200D3
:1002B000A095AA22A50E58F0A091A100A21509F0C0
:1002C000AA95AA0EA093A10048F04A2D08C0A091BB
:1002D000A100BA1608F0A395A093A1004FEF409398
:1002E00064007F7B485F08F07064A0916000A39574
:1002F000A093600059F0F894A9B7A160A9BF84FF4A
:1003000003C0A9B7A062A9BF3FBE1895A091740011
:10031000A395A093740041E050916800552329F003
:1003200085FF03C05A9550936800A0919600A130B4
:1003300018F0209299000DC020929A002092A300FC
:10034000A0919900AF5FA093990018F0AFEFA09330
:100350009900F894A9B7A160A9BF84FF03C0A9B709
:10036000A062A9BF3FBE18953FB646B557B58F7E70
:10037000A9B7A072A2118061A9B7AF7DA9BFA9B723
:10038000AE7FA9BF789481FD25C0AEB5AF7B96FD49
:10039000A064AEBD8260A6B396FDA095A0FF05C087
:1003A000409365005093660041C1AEB5A06496FDD0
:1003B000AF7BAEBDAA27A062A8BF8D7F85FF01C01D
:1003C00028C140E0A6B396FDA095A0FD22C14093B0
:1003D000960011C1AEB5A06496FDAF7BAEBD8D7F1A
:1003E00061FF72C0AEB5AF7B96FDA064AEBDAA271B
:1003F000A062A8BF82604093910050939200A090A9
:100400008F004A19B09090005B09BB24A22C4C3895
:10041000520518F42092950049C0A091D400AA2357
:1004200059F1483C520528F4A0E1BA2EAAE0AA2EC0
:1004300023C04836A1E05A0728F4A8E0BA2EAFE05E
:10044000AA2E1AC0403DA2E05A0728F4A4E0BA2E12
:10045000AEE1AA2E11C0403AA5E05A0728F4A2E066
:10046000BA2EACE3AA2E08C04839A8E05A0720F4F7
:10047000A1E0BA2EA8E7AA2EC42EA0919300CA1A12
:10048000D52EA0919400DA0ADD202AF4AFEFC094B3
:10049000D094CA1ADA0A20929500A8E0A210A0E02F
:1004A000CA14DA0618F4A1E0A093950040939300D3
:1004B00050939400409191005091920040938F008E
:1004C0005093900042E097C0A09165004A1BA09114
:1004D00066005A0B94FD82C093FD80C092FD7CC0E3
:1004E00086FF03C0D52EC42E0CC05695479591FDAE
:1004F00073C05695479590FD6FC0D52EC42ED694E7
:10050000C79461FD19C0AC2DAC51AD2DA24008F0CF
:1005100005C0DD2089F4AC2DA85C70F4A0916700C3
:10052000A395AA2311F0A0936700AA3008F471C024
:100530002092960081606DC0A0916700AA2319F0F7
:10054000AA95A0936700A22C5091BA0097FD06C00F
:10055000A090C800533011F4A090D000AAEFAA0ECA
:10056000A22DA21DCA18DA0A4FB74170533049F4C0
:10057000442321F087FD05C0806803C087FF01C0C8
:100580008F77442359F0533031F4AFEFC094D094B7
:10059000CA1ADA0A03C040E050E020C0533049F4E0
:1005A000CC0CDD1CAAE0CA1AD20818F4A0E0CA2EAE
:1005B000D22CAFEFCA16D20418F04FEF50E00EC0A5
:1005C000A091AC00CA9E412D000C441F50E008F0E1
:1005D00012C04FEF50E00FC05695479594FF07C0EB
:1005E000552309F04FEFA42FA6954A0F521D4F3FF8
:1005F000520508F04FEF40939600816061FF09C0FB
:10060000AFE1A095A923AB299A2F8F7DBB2009F4D8
:100610008062A8E1A093680085FF03C0AAE0A093D0
:10062000680061FD03C085FD01C08F7E85FD03C0AC
:10063000A6E0A0936900F894A9B7A160A9BF84FFC0
:1006400003C0A9B7A062A9BF3FBE189511E00AC0B8
:1006500013E008C01AE006C01EE104C014E602C0A0
:1006600018EC00C005E1BB27BA95F1F70A95D9F758
:100670001A95C1F708952AE338E709C020E33CE85A
:1006800006C02AE234EB03C025E238EC00C0B0918A
:10069000AD00BA9509F4089512E0BB27AD9ABA955A
:1006A000F1F7929ABA95F1F79298BA95F1F7AD9859
:1006B000BA95F1F7123009F0AC9A123009F4949A15
:1006C000B091AD00BA95F1F7123009F0AC98123044
:1006D00009F49498B7E8BA95F1F71A95F1F6022F54
:1006E000B22FBA95F1F70A95D9F73A9581F6AD9AF6
:1006F0000895221B39E0001F3A9509F40895221F3E
:10070000211B18F4210F8894F6CF0894F4CF622CA3
:10071000722CB0E08894B395221F331FE0F7379511
:1007200027958894912E802E020B130B10F4192D0F
:10073000082D10F4889401C00894661C771CBA95A3
:1007400071F7172D062D0895322D11232AF43A95AD
:1007500000951095031B130BF894029F712C002D2C
:10076000129F912C802C7894780C172D921C292D97
:10077000B4E06B2E2695179507956A94D9F7332325
:1007800021F000951095031B130B08950091B40000
:100790000430A1F1B0919600B15008F010C0B091B2
:1007A0006100B093630020927E0020927F0020922F
:1007B000800020928100209282006F7D1FC0609097
:1007C000B4006062B0916100B093620008E317EC7E
:1007D00020917A0030917B0036952795B62DBA95F9
:1007E00041F036952795B62DBA95BA9511F0369504
:1007F00027958DDF00937E0010937F000895009170
:100800007E00B09162000B1B10917F00120928F44A
:100810000038BFEF1B0740F009C00F37120508F47E
:1008200005C00FE710E002C000E81FEF009383004F
:1008300010938400089500918300B09180000B0F05
:1008400010918400B09181001B1F20E03091840042
:1008500033230AF42A95B09182002B1F1AF4203F0B
:1008600040F00AC02F3008F407C00FEF1FEF2FE051
:1008700003C000E010E020EF30916300B0919B00D6
:100880003B1718F4323030F009C0B0918400BB231C
:100890005AF004C0B0918400BB2332F4009380006E
:1008A000109381002093820008952091D700009139
:1008B0008300000F10918400111F46DF11232AF4DA
:1008C0000038BFEF1B0740F009C00F37120508F4CE
:1008D00005C00FE710E002C000E81FEF002352F050
:1008E000B0916200B01B0B2F18F0013008F00AC065
:1008F00001E008C000950F5FB09162000B0F08F097
:1009000001C00FEF0093850008952091D800009159
:1009100081001091820018DF11232AF40130BFEF0B
:100920001B0740F009C00F3F120508F405C00FEF88
:1009300010E002C001E01FEF112352F0B0918500DA
:10094000B01B0B2F18F0013008F00AC001E008C0FE
:1009500000950F5FB09185000B0F08F001C00FEFFD
:100960000093630008950FEF71FD1EC0B091D30096
:10097000BB23D1F0B0917B00BB23B1F00FEF1091FE
:100980007B00B7DEF894B091730072FDB5E00B9F69
:10099000112D002D7894112309F00FEFB0919E00D6
:1009A0000B1710F400919E0000939D000895009194
:1009B0007A0010917B0000541140B0919D0010F41A
:1009C000BA9501C0B39511F0B0939D00089500C091
:1009D00008952091B500B6B1B6FDFBCF04B115B1B5
:1009E000B6B1BF77B6B9B091AA00B395B093AA00DB
:1009F000B83060F12092AA00B091D200BB2321F15F
:100A0000112329F0B091AB00BF3F61F009C0B09154
:100A1000AB000B1739F020F4BB2321F0BA9502C0CC
:100A2000B395E1F300919B00B093AB00B03050F46C
:100A300000ECB03038F400E8B03020F400E4B0301E
:100A400008F400E000939B007F7E089510919B00C6
:100A5000B0E11B0F08F41FEF10939B00B091B4009E
:100A6000B43081F000919B00B0916300B01B10F492
:100A700000916300B0919D000B1708F00B2F502ED2
:100A800000936400B091AA00B73009F47061089532
:100A900002E3F894B091D9000B9F012D000C001FC8
:100AA0007894B0919B000B1710F000919B0000937D
:100AB000610000936300502E0093640000939E0039
:100AC000089520927A00B0EFB0937B000895F894D7
:100AD0000CB51DB52091740078943091750060902C
:100AE00076000093750010937600031B160971FDC4
:100AF00003C077FD80C028C07090770020937700F6
:100B00002709222319F00FEF1FEF0EC08090780005
:100B10009090790030937800609279000091750090
:100B2000109176000819190920917A0030917B0004
:100B300036952795020F131F10F40FEF1FEF009348
:100B40007A0010937B002BC020917A0030917B00BB
:100B50003901B4E08B2EB2E09B2E343040F08A9401
:100B60009A94383020F072FD02C08A949A94769458
:100B700067948A94E1F726193709992021F0169590
:100B800007959A94E1F7200F311F20937A00309354
:100B90007B0028F43FEF30937A0030937B003230B3
:100BA00008F4706871FF02C0B3E00DC0B091C400DA
:100BB00000917100023838F0B395003A08F0B3950F
:100BC000B63008F0B5E09B2EB4E08B2E10917B0080
:100BD00000917A0024E0169507952A95E1F7081907
:100BE000120928F0B02FB250B12FB20910F402E070
:100BF00010E0980126C020917A0030917B003901E5
:100C000076946794669466946694261932090695DC
:100C10000695200F321D20937A0030937B003230EE
:100C200008F07F7704E03695279536952795269529
:100C30002695201B10F0223008F422E089019090C4
:100C4000C40060FDFECFE0908B00F0908C006160EE
:100C5000B9B7B061B9BF380177FD41C076946794E8
:100C600000938B0010938C00B92DB330E1F0B0FDF0
:100C700004C0060D171D930106C0000F111F02507E
:100C8000120922E030E0B92DB33068F020938D00D6
:100C900030938E0000938700109388006092890043
:100CA00070928A003AC000938D0010938E002093BA
:100CB0008700309388006092890070928A0071FFEB
:100CC0000DC0BFE0B0938D0020928E00B0938900DC
:100CD00020928A00B0938B0020928C001EC06694F4
:100CE00000938B00B92DB33091F0B0FD03C0060D19
:100CF000262D03C0000F025022E0B92DB33038F08A
:100D000020938D00009387006092890006C00093B5
:100D10008D00209387006092890000917C0002FD85
:100D20000350013029F495FD0AC0B6E0B7B909C0F7
:100D3000023019F4B7E0B7B904C095FDF6CFB0E0C2
:100D4000B7B90091A200000F10F4BBE60B27009387
:100D5000A20060FDFECFB2E0B0936E006160B9B753
:100D6000B061B9BFB72FB670D1F020917A00309141
:100D70007B00369527953695279571FF02C0B0E424
:100D80003B0FF8940CB51DB5020F131F1BBD0ABD18
:100D90006160B0E1B8BFB9B7B061B9BF78940895E8
:100DA000686020927D0020E066FD20E206C0686059
:100DB00020927D0020E266FD20E001E011E077FD59
:100DC00011C0B72FB67009F0677F14E100917B0066
:100DD000069509F403950F3008F00FE071FF02C08B
:100DE00004E114E160FD0FC0B0917D00BB2359F018
:100DF00071FF06C0B0916E00BA95B0936E0011F409
:100E000070624FC0ABDFB0B7B77FB0BFB8B1B0B79B
:100E1000B860B0BFB0917D00B395B0937D00B8B11C
:100E200077FD06C0B1E071FDB3E0BA95F1F7B8B156
:100E3000B072B21709F02AC071FF05C003950117FF
:100E400008F00A95CFCF63FD05C00395011708F0A0
:100E5000B4CFC8CF677FF8943CB56DB470907A007A
:100E6000B0917B00770CBB1F08F4BFEF770CBB1F62
:100E700008F4BFEF370D6B1E6BBC3ABD6160B0E18B
:100E8000B8BFB9B7B061B9BF789497CFB0916D00D2
:100E9000B13008F492CF63FD90CF0A9509F0A2CF4C
:100EA0007F7D20918D0030918E00F894B0E1B8BF25
:100EB0000CB51DB5020F131F1BBD0ABDE0908700C6
:100EC000F09088006160B9B7B061B9BF7894B72F6E
:100ED000B67039F0B0916D0072FFB395B0936D00AC
:100EE00009C075FF07C066FD05C063FD03C0BF9163
:100EF000BF91FBC4089500E063FF01C001E0F894D6
:100F000010917100B7E01B9F212D102D7894200FB8
:100F10002695179526951795269517951093710088
:100F2000183718F4B8E7B093710000917100B091D0
:100F300072000B1720F06061AC989298949860FD55
:100F4000FECFE0908900F0908A006160B9B7B0618F
:100F5000B9BF0895B2E095FD0AC0F894B0937C0043
:100F6000AD9A959862FF01C0949A7894F4C0F89471
:100F7000B0937C00AD9A939862FF01C0AC9A7894CC
:100F8000EAC0B3E082FF24C095FD11C002E0F894EE
:100F9000B0937C00E1E8F0E00093B1009498939A5C
:100FA00062FF02C0929A01C0AD987894D4C002E06A
:100FB000F894B0937C00E1E8F0E00093B100AC98C5
:100FC000959A62FF02C0929A01C0AD987894C3C00E
:100FD00095FD0BC0F894B0937C00EBE6F0E094989C
:100FE00062FF01C0929A7894B6C0F894B0937C00E6
:100FF000EBE6F0E0AC9862FF01C0929A7894ABC047
:10100000B4E095FD0AC0F894B0937C00959A93984B
:1010100062FF01C0929A78949EC0F894B0937C00CD
:10102000939A959862FF01C0929A789494C0B5E023
:1010300082FF24C095FD11C001E0F894B0937C00BC
:10104000E7E7F0E00093B1009298AD9A62FF02C02A
:10105000AC9A01C0959878947EC004E0F894B0935F
:101060007C00EBE8F0E00093B1009298AD9A62FF4B
:1010700002C0949A01C0939878946DC095FD0BC0FE
:10108000F894B0937C00E5E6F0E0929862FF01C02E
:10109000AC9A789460C0F894B0937C00E1E7F0E0FB
:1010A000929862FF01C0949A789455C0B6E095FD7D
:1010B0000AC0F894B0937C00939AAD9862FF01C087
:1010C000AC9A789448C0F894B0937C00959AAD9807
:1010D00062FF01C0949A78943EC0B1E082FF24C0C0
:1010E00095FD11C004E0F894B0937C00EBE8F0E0CB
:1010F0000093B100AC98959A62FF02C0949A01C027
:101100009398789428C001E0F894B0937C00E7E7C6
:10111000F0E00093B1009498939A62FF02C0AC9AF9
:1011200001C09598789417C095FD0BC0F894B093C2
:101130007C00E1E7F0E0AC9862FF01C0949A7894FB
:101140000AC0F894B0937C00E5E6F0E0949862FF62
:1011500001C0AC9A78946F7E089524E630E0F901DE
:101160002092B100AC9892989498959AAD9A939ADF
:101170006B7F0895A2EBB0E009E00D9309E00D93B9
:1011800004E00D930FEF0D9303E00D930FEF0D931C
:101190000BE00D9303E00D9301E00D9301E00D933F
:1011A000AEEBB0E001E00D930FEF0D930D930D93B7
:1011B0000D930D9303E00D930FEF0D930FEF0D9330
:1011C0000D9305E20D9300ED0D9308E20D9300E5FC
:1011D0000D9304E00D930FEF0D9302E00D9300E0EB
:1011E0000D930AE70D930FEF0D9300E00D9301E0CF
:1011F0000D9300E00D9303E00D9300E00D9308952F
:101200002091B9008B7F233009F48460B091BA003B
:10121000B33019F09F7DB1FD90629F7BB091BB0010
:10122000B1FD9064223011F0886001C0877F08957D
:101230000A95E00FF21DB4910895ECE1F0E0009101
:10124000B200F6DFB093D700ECE1F0E00091B3001C
:10125000EFDFB093D800EAE2F0E00091B800E8DFF9
:10126000B093D9000091B800023008F402E0009376
:101270007300B091CE000FEFB23009F400EAB33042
:1012800009F402E800937200E8E3F0E00091D50071
:10129000CFDFB093A000089508952091C800309149
:1012A000C900B091BA00B33009F43E5097FF02C0B4
:1012B00020E03FEFB32FB21B6B2EB25810F4B2E810
:1012C0006B2E00E00395609EB12DBD57D8F30093BF
:1012D000AC0008959068E1DFBFD9BED920E030E0CE
:1012E000B0E16B2EB5D9B09196002B0F321D6A94E8
:1012F000C9F7B4E036952795BA95E1F7822E9F7726
:10130000CCDF0895F894E3E0F0E0B9E0B7BFB49122
:10131000B078C1F3F894A895B1B5B861B1BDB0E0AB
:10132000B1BDB4E0BEBFBFE5BDBF17DFB0E0B8BB25
:10133000B0E1B7BBB0E2B5BBB0E3B4BBB8E2B2BB9F
:10134000BCE3B1BB2224A0E0B0E02D92AA31E9F7C2
:10135000A0E6B0E00FEF2D920A95E9F7B1E0B09367
:10136000A20008DFFAD2B6B1B460B6B90091CA00E3
:101370000093AD00B1E0B0936A00F89471D97BD9C5
:101380006BD97CD969D97DD967D9F8940AEF1AEF5E
:10139000A6B396FDA095A0FF1FC01A95C9F70A95A0
:1013A000B1F7E0E0FCE1B591B43E39F4B591B03E5F
:1013B00021F4B591BF3F09F40CC0E0E0F395F3953B
:1013C000B591B83F49F4B591B43931F4B591BA3A11
:1013D00019F4EE27F695099413DF2FDF5DDF5DDF4B
:1013E0000091CA000093AD00B8DEB2E0B3BFB2E036
:1013F000BEBDB2E0B5BDB1E5B8BFB9BFB0B7B77F4C
:10140000B0BFB8B1B0B7B860B0BF20D97894DFDA58
:1014100020927000BEB5B06496FDBF7BBEBDB9B76B
:10142000B062B9BFBB27B062B8BF8D7F19D9626007
:1014300033E02CE0B0919500BB2321F42CE03A95E9
:1014400009F4A3CF09D980FFA0CF8E7FB091960079
:10145000B23078F3B92FBF710091980000939700D4
:10146000B0939800B01729F72A9521F76D7FBEB584
:10147000B06496FDBF7BBEBDBB27B062B8BF8D7F99
:10148000B091D400BB2321F48062B92FB0709B2FA0
:101490008F7B20926700E2D885FF05C0B09167007E
:1014A000BA3008F08064D4D802E085FF01C000E0C3
:1014B000B0919600B017B8F3F894DDD8DCD8DBD83B
:1014C0007894CED820928600B091BA00B33009F457
:1014D0007DC0BED8B091BE00B13008F477C0B091E5
:1014E0006A00B13008F472C085FD18C0B091960052
:1014F000BF3F08F46BC0F894C7D87894AFD8B091C8
:101500009600B130C0F7F894B6D8A4D8B4D878947F
:10151000A5D8B0919600BF3FB0F3E0C2B3E09B2ED8
:101520009068F894BADE789499D8F8949F77B5DEED
:1015300080909600B0919600BF37789408F44EC022
:1015400085D8F894A1D878949A9451F7C3DEB82D31
:10155000B093C90085D8F89494D27894BAE09B2EC1
:101560009068F8949ADE789479D8F8949F7795DE0D
:1015700080909600B0919600BF37789478F766D83F
:10158000F89479D867D877D878949A9449F7A2DEF6
:10159000B82DBB5FB093C8000B2F1091C900125833
:1015A00010F0100B20F4B2E80B0F0093C90058D8CC
:1015B000F89400D275D2789451D8F8946EDE78946D
:1015C000B0919600BF3F08F48FCF88C2009196007B
:1015D000B09186000B1710F0009386003FD801E011
:1015E000B091BA00B35009F405E0B0919600B0177D
:1015F00008F06ACFF89448D847D846D8789430D8BD
:1016000020926A0020926B0020926C00B0916B00D7
:10161000B395B0936B00BF3F71F5B0916C00B3957B
:10162000B0936C00B091CC0009E1BA9559F002E397
:10163000BA9541F00DE7BA9529F00AEFBA9511F085
:1016400020926C00B0916C00B017A8F086DDFED738
:10165000B0916C00BA95B0936C0020926B00B09181
:10166000CB00B093AD00F8940FD87894B091CA0035
:10167000B093AD00F3D7EED7B0916800BB2319F457
:1016800085FF01C082CE01E085FD01C006E0B0917A
:101690009600B01708F4BACFB091BA00B35009F071
:1016A000DDD7B0916800BB2309F46FCEF89455DD07
:1016B000209261002092620020926300522C2092BE
:1016C00064002092A1007894B091B700BB0FB09352
:1016D0009F0020927E0020927F0020928000209226
:1016E0008100209282002092AA0060E070E02092A7
:1016F0007100B8E0B093AA007061A8D7B2E074FDA1
:10170000B2E0B7B9B6B1B068B064B6B9B6B1B6FDBB
:10171000FDCF04B115B1B6B1BF77B6B9112309F049
:101720000FEF0093AB0055D9B8E0B093AA007061F9
:1017300067DDF894BFEFB0939B00AAD9B091610028
:10174000B0939B00B0939C00B0939D007894B1E05F
:10175000B0936100B09363005B2EB0936400B093CC
:10176000A400B0919A00B093A300B091BA00B33036
:1017700019F49F7D87FD90627160726020926D0008
:1017800095DCABDC9ED9A3D99CD9A1D99AD90FDB22
:10179000FDD7B1DBDFDB9BD903DB65FD30D877FFFD
:1017A000E2D877FD04D9A7DBECDB91D900DB65FD3E
:1017B00042D8A1DB25DC8BD9F3DA65FD76D89BDB3B
:1017C00036DC85D9F4DA65FDA0D895DB6FDC7FD9EE
:1017D000E7DAB2E074FDB2E0B7B9B6B1B068B064B0
:1017E000B6B989DB7ADC73D9F4D871FF24C0B09123
:1017F0009E00B0939B00B0939C00B0919A00B09370
:10180000A300B1E0B093A40018E12CE0B0916D000A
:10181000B11758F07D7F746020936F00B0919E00E7
:10182000B0939B00B0939D0006C0B0919600B1307C
:1018300008F0ADCF64C072FF15C066FD13C0B09153
:101840006F00BA9519F47B7F7860A1CFB0936F00D9
:10185000B0919600B13008F09ACFB091BA00B33091
:1018600009F04DC020927000B09199000AEF1091DC
:10187000D600112309F003E0B01708F040C085FF3F
:1018800004C0B0916800BB23D1F1B091BA00B3306D
:1018900081F495FD03C087FD04C00BC087FF01C024
:1018A00008C066FD06C06064B0919E00B0939B00C6
:1018B00083CF00EF66FF05C0B0919E00B0939B0000
:1018C00000E2B0917B00B01708F461CF66FF17C04B
:1018D0006F7B9F7D87FD90627460B2E1B0936F0073
:1018E000B0919E00B0939B0052CFB0917000B39521
:1018F000B0937000B0919600BB2309F002C0209213
:101900007000F8942ADC8090B900B2E0B093B9007E
:1019100077DC8092B90020926100209262002092D0
:101920006300522C2092640020929F0060E070E0DF
:10193000789494D612DC0091D600002319F0AC9A6A
:10194000929A949AB6B1B460B6B985FF05C0B091C9
:101950007000B43008F019CD55CEEDE0F0E023D0A2
:10196000053509F01BC0EEE0F0E01DD00A3A09F0A1
:1019700015C03AE0A2EBB0E0E3E0F0E014D00D9344
:1019800031963A95D9F739E1AEEBB0E0EFE0F0E00F
:101990000AD00D9331963A95D9F702C0EBDB0AD005
:1019A000E8E2F0E00895E199FECFEEBBFFBBE09ADC
:1019B0000DB308951ED03AE0A2EBB0E0E3E0F0E012
:1019C0000D910FD031963A95D9F739E1AEEBB0E0F1
:1019D000EFE0F0E00D9105D031963A95D9F712D0AD
:1019E0000895E199FECF0DBBEEBBFFBBE29AE19AF1
:1019F0000895EDE0F0E00FEFF4DFEEE0F0E00FEF40
:101A0000F0DF0895EDE0F0E005E5EBDFEEE0F0E07B
:101A10000AEAE7DF08953091AE000091AF0031305F
:101A200011F40093B200323011F40093B30033305C
:101A300011F40093B400343011F40093B600353043
:101A400011F40093B800363011F40093C40037301D
:101A500011F40093B900383011F40093D5003930F7
:101A600011F40093CE003A3011F40093BA003B30E9
:101A700011F40093BB00089525E0F2D52A95E9F70B
:101A80000895F9D5FBD5FDD5FFD5E4D5F4D5F6D528
:101A9000F8D5FAD5DFD5EFD5F1D5F3D5F5D508953D
:101AA000F3D5EFD5EBD5E7D5D5D5EED5EAD5E6D547
:101AB000E2D5D0D5E9D5E5D5E1D5DDD5089580903D
:101AC000AE009090AF00D7D5D6D5D5D5C3D58A94E2
:101AD000D1F7DAD5BFD59A94E1F70895F894D1DF1C
:101AE0007894CADFC9DFB1E0B093AE00B1E0B09343
:101AF000AF002092B000F894E2DF7894B5E06B2E4E
:101B000070909600ADD5B09196007B16C9F7B130B4
:101B100018F0BF3F40F107C07EDFF8944BDFB1DF24
:101B2000B8E0B1BDA9DF6A9459F7B091B000B395A0
:101B3000B093B000B33008F4DECF9EDFB091AF00B9
:101B4000B395B093AF00F894B091AE00BA95EEE3C0
:101B5000F0E0EB0FF21D049178940395B091AF0083
:101B6000B01708F4C6CF88DF87DFB091AE00B39519
:101B7000B093AE00B091AE00BC3008F4B7CFFADA43
:0C1B8000F89418DFB8E0B1BD77DFBCCBF3
:00000001FF
